BL51 BANKED LINKER/LOCATER V6.22                                                        01/27/2016  22:38:18  PAGE 1


BL51 BANKED LINKER/LOCATER V6.22, INVOKED BY:
C:\KEIL\C51\BIN\BL51.EXE LQ12864.obj, LQ12864main.obj TO LQ_OLED RAMSIZE (256)


MEMORY MODEL: SMALL


INPUT MODULES INCLUDED:
  LQ12864.obj (LQ12864)
  LQ12864main.obj (LQ12864MAIN)
  C:\KEIL\C51\LIB\C51S.LIB (?C_STARTUP)
  C:\KEIL\C51\LIB\C51S.LIB (?C?CLDOPTR)
  C:\KEIL\C51\LIB\C51S.LIB (?C_INIT)


LINK MAP OF MODULE:  LQ_OLED (LQ12864)


            TYPE    BASE      LENGTH    RELOCATION   SEGMENT NAME
            -----------------------------------------------------

            * * * * * * *   D A T A   M E M O R Y   * * * * * * *
            REG     0000H     0008H     ABSOLUTE     "REG BANK 0"
            DATA    0008H     0070H     UNIT         ?DT?LQ12864
            DATA    0078H     0008H     UNIT         _DATA_GROUP_
            IDATA   0080H     0001H     UNIT         ?STACK

            * * * * * * *   C O D E   M E M O R Y   * * * * * * *
            CODE    0000H     0003H     ABSOLUTE     
            CODE    0003H     0818H     UNIT         ?CO?LQ12864
            CODE    081BH     009FH     UNIT         ?PR?LCD_INIT?LQ12864
            CODE    08BAH     008FH     UNIT         ?PR?_LCD_P8X16STR?LQ12864
            CODE    0949H     008CH     UNIT         ?C_C51STARTUP
            CODE    09D5H     007BH     UNIT         ?PR?MAIN?LQ12864MAIN
            CODE    0A50H     0074H     UNIT         ?C_INITSEG
            CODE    0AC4H     0064H     UNIT         ?PR?_LCD_P6X8STR?LQ12864
            CODE    0B28H     0044H     UNIT         ?PR?_LCD_P14X16CH?LQ12864
            CODE    0B6CH     0035H     UNIT         ?PR?_DELAY?LQ12864MAIN
            CODE    0BA1H     002EH     UNIT         ?PR?_LCD_WRCMD?LQ12864
            CODE    0BCFH     002DH     UNIT         ?C?LIB_CODE
            CODE    0BFCH     0026H     UNIT         ?PR?_LCD_WRDAT?LQ12864
            CODE    0C22H     0021H     UNIT         ?CO?LQ12864MAIN
            CODE    0C43H     001CH     UNIT         ?PR?_LCD_SET_POS?LQ12864
            CODE    0C5FH     001AH     UNIT         ?PR?_LCD_DLY_MS?LQ12864
            CODE    0C79H     0018H     UNIT         ?PR?_LCD_FILL?LQ12864
            CODE    0C91H     0016H     UNIT         ?PR?LCD_CLS?LQ12864



OVERLAY MAP OF MODULE:   LQ_OLED (LQ12864)


SEGMENT                             DATA_GROUP 
  +--> CALLED SEGMENT             START    LENGTH
-------------------------------------------------
?C_C51STARTUP                     -----    -----
  +--> ?PR?MAIN?LQ12864MAIN
  +--> ?C_INITSEG
BL51 BANKED LINKER/LOCATER V6.22                                                      01/27/2016  22:38:18  PAGE 2



?PR?MAIN?LQ12864MAIN              0078H    0001H
  +--> ?PR?LCD_INIT?LQ12864
  +--> ?PR?_LCD_FILL?LQ12864
  +--> ?PR?_DELAY?LQ12864MAIN
  +--> ?PR?_LCD_P14X16CH?LQ12864
  +--> ?CO?LQ12864MAIN
  +--> ?PR?_LCD_P8X16STR?LQ12864
  +--> ?PR?_LCD_P6X8STR?LQ12864
  +--> ?PR?LCD_CLS?LQ12864

?PR?LCD_INIT?LQ12864              -----    -----
  +--> ?PR?_LCD_DLY_MS?LQ12864
  +--> ?PR?_LCD_WRCMD?LQ12864
  +--> ?PR?_LCD_FILL?LQ12864
  +--> ?PR?_LCD_SET_POS?LQ12864

?PR?_LCD_FILL?LQ12864             -----    -----
  +--> ?PR?_LCD_WRCMD?LQ12864
  +--> ?PR?_LCD_WRDAT?LQ12864

?PR?_LCD_SET_POS?LQ12864          -----    -----
  +--> ?PR?_LCD_WRCMD?LQ12864

?PR?_LCD_P14X16CH?LQ12864         0079H    0002H
  +--> ?PR?_LCD_SET_POS?LQ12864
  +--> ?PR?_LCD_WRDAT?LQ12864

?PR?_LCD_P8X16STR?LQ12864         0079H    0007H
  +--> ?PR?_LCD_SET_POS?LQ12864
  +--> ?CO?LQ12864
  +--> ?PR?_LCD_WRDAT?LQ12864

?PR?_LCD_P6X8STR?LQ12864          0079H    0007H
  +--> ?PR?_LCD_SET_POS?LQ12864
  +--> ?CO?LQ12864
  +--> ?PR?_LCD_WRDAT?LQ12864

?PR?LCD_CLS?LQ12864               -----    -----
  +--> ?PR?_LCD_WRCMD?LQ12864
  +--> ?PR?_LCD_WRDAT?LQ12864



SYMBOL TABLE OF MODULE:  LQ_OLED (LQ12864)

  VALUE           TYPE          NAME
  ----------------------------------

  -------         MODULE        LQ12864
  C:0000H         SYMBOL        _ICE_DUMMY_
  D:0090H         PUBLIC        P1
  D:0008H         PUBLIC        F14x16
  B:0090H.1       PUBLIC        LCD_SDA
  D:00A8H         PUBLIC        IE
  C:0BAEH         PUBLIC        _LCD_WrCmd
  C:0C91H         PUBLIC        LCD_CLS
BL51 BANKED LINKER/LOCATER V6.22                                                      01/27/2016  22:38:18  PAGE 3


  B:0090H.0       PUBLIC        LCD_SCL
  C:0C01H         PUBLIC        _LCD_WrDat
  D:00B8H         PUBLIC        IP
  D:00D8H         PUBLIC        CCON
  C:0AC4H         PUBLIC        _LCD_P6x8Str
  C:0003H         PUBLIC        F6x8
  B:0090H.2       PUBLIC        LCD_RST
  D:0098H         PUBLIC        SCON
  D:0088H         PUBLIC        TCON
  B:0090H.3       PUBLIC        LCD_DC
  C:0C79H         PUBLIC        _LCD_Fill
  C:022BH         PUBLIC        F8X16
  C:081BH         PUBLIC        LCD_Init
  C:08BAH         PUBLIC        _LCD_P8x16Str
  C:0C5FH         PUBLIC        _LCD_DLY_ms
  C:0C43H         PUBLIC        _LCD_Set_Pos
  C:0B28H         PUBLIC        _LCD_P14x16Ch
  D:00D0H         PUBLIC        PSW
  C:0BFCH         SYMBOL        L?0061
  -------         PROC          L?0060
  -------         ENDPROC       L?0060
  C:0BFCH         SYMBOL        L?0061
  -------         PROC          _LCD_WRDAT
  D:0007H         SYMBOL        dat
  -------         DO            
  D:0006H         SYMBOL        i
  -------         ENDDO         
  C:0C01H         LINE#         289
  C:0C01H         LINE#         290
  C:0C01H         LINE#         291
  C:0C03H         LINE#         293
  C:0C05H         LINE#         294
  C:0C07H         LINE#         296
  C:0C0DH         LINE#         297
  C:0C0DH         LINE#         298
  C:0C15H         LINE#         299
  C:0C17H         LINE#         300
  C:0C19H         LINE#         303
  C:0C1BH         LINE#         304
  C:0C1FH         LINE#         305
  C:0C21H         LINE#         307
  -------         ENDPROC       _LCD_WRDAT
  C:0BA9H         SYMBOL        L?0059
  -------         PROC          L?0058
  -------         ENDPROC       L?0058
  C:0BA9H         SYMBOL        L?0059
  -------         PROC          _LCD_WRCMD
  D:0007H         SYMBOL        cmd
  -------         DO            
  D:0006H         SYMBOL        i
  -------         ENDDO         
  C:0BAEH         LINE#         308
  C:0BAEH         LINE#         309
  C:0BAEH         LINE#         310
  C:0BB0H         LINE#         313
  C:0BB2H         LINE#         314
  C:0BB4H         LINE#         316
BL51 BANKED LINKER/LOCATER V6.22                                                      01/27/2016  22:38:18  PAGE 4


  C:0BBAH         LINE#         317
  C:0BBAH         LINE#         318
  C:0BC2H         LINE#         319
  C:0BC4H         LINE#         320
  C:0BC6H         LINE#         323
  C:0BC8H         LINE#         324
  C:0BCCH         LINE#         325
  C:0BCEH         LINE#         327
  -------         ENDPROC       _LCD_WRCMD
  -------         PROC          _LCD_SET_POS
  D:0004H         SYMBOL        x
  D:0005H         SYMBOL        y
  C:0C43H         LINE#         328
  C:0C45H         LINE#         329
  C:0C45H         LINE#         330
  C:0C4CH         LINE#         331
  C:0C58H         LINE#         332
  -------         ENDPROC       _LCD_SET_POS
  -------         PROC          _LCD_FILL
  D:0004H         SYMBOL        bmp_dat
  -------         DO            
  D:0003H         SYMBOL        y
  D:0002H         SYMBOL        x
  -------         ENDDO         
  C:0C79H         LINE#         334
  C:0C7BH         LINE#         335
  C:0C7BH         LINE#         338
  C:0C7DH         LINE#         339
  C:0C7DH         LINE#         340
  C:0C7EH         LINE#         341
  C:0C7EH         LINE#         342
  C:0C81H         LINE#         343
  C:0C83H         LINE#         344
  C:0C8CH         LINE#         345
  C:0C90H         LINE#         346
  -------         ENDPROC       _LCD_FILL
  -------         PROC          LCD_CLS
  -------         DO            
  D:0004H         SYMBOL        y
  D:0003H         SYMBOL        x
  -------         ENDDO         
  C:0C91H         LINE#         347
  C:0C91H         LINE#         348
  C:0C91H         LINE#         350
  C:0C93H         LINE#         351
  C:0C93H         LINE#         352
  C:0C94H         LINE#         353
  C:0C94H         LINE#         354
  C:0C97H         LINE#         355
  C:0C99H         LINE#         356
  C:0CA2H         LINE#         357
  C:0CA6H         LINE#         358
  -------         ENDPROC       LCD_CLS
  -------         PROC          _LCD_DLY_MS
  D:0006H         SYMBOL        ms
  -------         DO            
  D:0004H         SYMBOL        a
BL51 BANKED LINKER/LOCATER V6.22                                                      01/27/2016  22:38:18  PAGE 5


  -------         ENDDO         
  C:0C5FH         LINE#         359
  C:0C5FH         LINE#         360
  C:0C5FH         LINE#         362
  C:0C63H         LINE#         363
  C:0C63H         LINE#         364
  C:0C67H         LINE#         365
  C:0C71H         LINE#         366
  C:0C76H         LINE#         367
  C:0C78H         LINE#         369
  -------         ENDPROC       _LCD_DLY_MS
  -------         PROC          LCD_INIT
  C:081BH         LINE#         370
  C:081BH         LINE#         371
  C:081BH         LINE#         372
  C:081DH         LINE#         374
  C:081FH         LINE#         375
  C:0826H         LINE#         376
  C:0828H         LINE#         380
  C:082DH         LINE#         381
  C:082FH         LINE#         382
  C:0832H         LINE#         383
  C:0837H         LINE#         384
  C:083CH         LINE#         385
  C:0841H         LINE#         386
  C:0846H         LINE#         387
  C:084BH         LINE#         388
  C:0850H         LINE#         389
  C:0855H         LINE#         390
  C:085AH         LINE#         391
  C:085FH         LINE#         392
  C:0864H         LINE#         393
  C:0869H         LINE#         394
  C:086EH         LINE#         395
  C:0873H         LINE#         396
  C:0878H         LINE#         397
  C:087DH         LINE#         398
  C:0882H         LINE#         399
  C:0887H         LINE#         400
  C:088CH         LINE#         401
  C:0891H         LINE#         402
  C:0896H         LINE#         403
  C:089BH         LINE#         404
  C:08A0H         LINE#         405
  C:08A5H         LINE#         406
  C:08AAH         LINE#         407
  C:08AFH         LINE#         408
  C:08B4H         LINE#         409
  -------         ENDPROC       LCD_INIT
  -------         PROC          _LCD_P6X8STR
  D:0079H         SYMBOL        x
  D:007AH         SYMBOL        y
  D:007BH         SYMBOL        ch
  -------         DO            
  D:007EH         SYMBOL        c
  D:0004H         SYMBOL        i
  D:007FH         SYMBOL        j
BL51 BANKED LINKER/LOCATER V6.22                                                      01/27/2016  22:38:18  PAGE 6


  -------         ENDDO         
  C:0AC4H         LINE#         418
  C:0ACEH         LINE#         419
  C:0ACEH         LINE#         420
  C:0AD4H         LINE#         421
  C:0AE5H         LINE#         422
  C:0AE5H         LINE#         423
  C:0AE9H         LINE#         424
  C:0AF5H         LINE#         425
  C:0AFCH         LINE#         426
  C:0AFEH         LINE#         427
  C:0B1DH         LINE#         428
  C:0B23H         LINE#         429
  C:0B25H         LINE#         430
  C:0B27H         LINE#         431
  -------         ENDPROC       _LCD_P6X8STR
  -------         PROC          _LCD_P8X16STR
  D:0079H         SYMBOL        x
  D:007AH         SYMBOL        y
  D:007BH         SYMBOL        ch
  -------         DO            
  D:007EH         SYMBOL        c
  D:0004H         SYMBOL        i
  D:007FH         SYMBOL        j
  -------         ENDDO         
  C:08BAH         LINE#         439
  C:08C4H         LINE#         440
  C:08C4H         LINE#         441
  C:08CAH         LINE#         443
  C:08DBH         LINE#         444
  C:08DBH         LINE#         445
  C:08DFH         LINE#         446
  C:08EBH         LINE#         447
  C:08F2H         LINE#         448
  C:08F4H         LINE#         449
  C:0913H         LINE#         450
  C:091CH         LINE#         451
  C:091EH         LINE#         452
  C:093DH         LINE#         453
  C:0943H         LINE#         454
  C:0945H         LINE#         455
  C:0948H         LINE#         456
  -------         ENDPROC       _LCD_P8X16STR
  -------         PROC          _LCD_P14X16CH
  D:0079H         SYMBOL        x
  D:0002H         SYMBOL        y
  D:0003H         SYMBOL        N
  -------         DO            
  D:0004H         SYMBOL        wm
  D:007AH         SYMBOL        ii
  D:0082H         SYMBOL        adder
  -------         ENDDO         
  C:0B28H         LINE#         459
  C:0B2CH         LINE#         460
  C:0B2CH         LINE#         461
  C:0B30H         LINE#         462
  C:0B3AH         LINE#         463
BL51 BANKED LINKER/LOCATER V6.22                                                      01/27/2016  22:38:18  PAGE 7


  C:0B3FH         LINE#         464
  C:0B41H         LINE#         465
  C:0B41H         LINE#         466
  C:0B4CH         LINE#         467
  C:0B4DH         LINE#         468
  C:0B51H         LINE#         469
  C:0B59H         LINE#         470
  C:0B5BH         LINE#         471
  C:0B5BH         LINE#         472
  C:0B66H         LINE#         473
  C:0B67H         LINE#         474
  C:0B6BH         LINE#         475
  -------         ENDPROC       _LCD_P14X16CH
  -------         ENDMOD        LQ12864

  -------         MODULE        LQ12864MAIN
  C:0000H         SYMBOL        _ICE_DUMMY_
  D:00A8H         PUBLIC        IE
  C:0B6CH         PUBLIC        _delay
  D:00B8H         PUBLIC        IP
  D:00D8H         PUBLIC        CCON
  C:09D5H         PUBLIC        main
  D:0098H         PUBLIC        SCON
  D:0088H         PUBLIC        TCON
  D:00D0H         PUBLIC        PSW
  -------         PROC          _DELAY
  D:0006H         SYMBOL        ms
  -------         DO            
  D:0004H         SYMBOL        ii
  D:0002H         SYMBOL        jj
  -------         ENDDO         
  C:0B6CH         LINE#         21
  C:0B6CH         LINE#         22
  C:0B6CH         LINE#         24
  C:0B7BH         LINE#         25
  C:0B8BH         LINE#         26
  C:0BA0H         LINE#         28
  -------         ENDPROC       _DELAY
  -------         PROC          MAIN
  -------         DO            
  D:0078H         SYMBOL        i
  -------         ENDDO         
  C:09D5H         LINE#         31
  C:09D5H         LINE#         32
  C:09D5H         LINE#         33
  C:09D8H         LINE#         35
  C:09DBH         LINE#         36
  C:09DBH         LINE#         37
  C:09DBH         LINE#         38
  C:09E0H         LINE#         39
  C:09E7H         LINE#         40
  C:09ECH         LINE#         41
  C:09F3H         LINE#         42
  C:09FBH         LINE#         43
  C:0A04H         LINE#         44
  C:0A0DH         LINE#         45
  C:0A16H         LINE#         46
BL51 BANKED LINKER/LOCATER V6.22                                                      01/27/2016  22:38:18  PAGE 8


  C:0A23H         LINE#         47
  C:0A30H         LINE#         48
  C:0A3DH         LINE#         49
  C:0A44H         LINE#         50
  C:0A47H         LINE#         52
  C:0A4EH         LINE#         70
  -------         ENDPROC       MAIN
  -------         ENDMOD        LQ12864MAIN

  -------         MODULE        ?C?CLDOPTR
  C:0BCFH         PUBLIC        ?C?CLDOPTR
  -------         ENDMOD        ?C?CLDOPTR

Program Size: data=129.0 xdata=0 code=3239
LINK/LOCATE RUN COMPLETE.  0 WARNING(S),  0 ERROR(S)
